:020000000528D1
:1000080052298B138312031383120313850186016C
:100018008316FF30831603138500FF308600831292
:100028008B13063083120313A000A101A2018730AD
:1000380083168316031381008312C33083120313BC
:10004800D400D5018100A0308B00D601FF30D90142
:10005800DA01DB00DC00892883120313D8000310BF
:10006800560D593E8400831357088000840A5808A7
:100078008000D60A5608013A0319D6010310560D16
:100088008313593E84000008840A000403193D289C
:10009800801B3D2800088A00840300088200831220
:1000A80003130508C7002730C9001030C8004808E6
:1000B8004904031D6028782883120313470805069E
:1000C8004605003A031D69287128831203130508A1
:1000D800C7002730C9001030C800FF30C807031810
:1000E800C90AFF30C9075B2883120313470846056E
:1000F800003A03090439031D0130C3008328831221
:10010800031345088A0044088200831203138501FB
:10011800FE30831603138500831203138601FF3014
:100128008316031386000730831203139F00BA0156
:10013800BB01BC01BD010330BE0003110319A52892
:10014800A6284C29831203138501B8013E08BF0075
:100158000310BF0D3F08FF3EBF003808803AFC007F
:100168003F08803A7C02031CBA28E1288312031353
:10017800B401B501B601B701031437083604031DED
:10018800CD2827303502031CCD28031DCD2810307B
:100198003402031CD028DB2883120313B901B40AE4
:1001A8000319B50A0319B60A0319B70AC02801309A
:1001B800831203138506B80AAA2883120313B4010D
:1001C800B501B601B701031437083604031DF42836
:1001D8009C303502031CF428031DF42840303402F7
:1001E800031CF728022983120313B901B40A03195F
:1001F800B50A0319B60A0319B70AE728403083126B
:100208000313C6000130C5000E30C40000308A0058
:1002180053308200831203134308BA003A083B069E
:10022800031D1729282983120313BA0803191D2946
:100238002629FF3083120313BE07FF30BE0707309D
:10024800BE05BE0A3A08BB008030C6000130C500B2
:100258003230C40000308A00533082008312031306
:100268004308BC003C083D06031D3B294B2983126B
:100278000313BC08031941294929FF3083120313CA
:10028800BE07BE0A0730BE05BE0A3C08BD00A1284D
:100298008312031333088A0032088200FF00030E1A
:1002A8008312031383120313CE00CE0E0A08CF0065
:1002B8000408D0000B1D7129540881005030D5075F
:1002C800B4300318013EFF3A013ED4000B11FF3051
:1002D800DC1B7129DB07031CDC077C08D1007D08C7
:1002E800D2007E08D3005308FE005208FD005108D2
:1002F800FC00500884004F088A004E088300FF0E57
:040308007F0E09005B
:02400E00103F61
:00000001FF
